:100000000C945F010C9497010C9497010C94970148
:100010000C9497010C9497010C9497010C94970100
:100020000C9497010C9497010C941D1A0C94EF1AE0
:100030000C9478150C9497010C9497010C949701EB
:100040000C9497010C9497010C9497010C949701D0
:100050000C9497010C9400160C9497010C94970142
:100060000C9497010C9497010C9497010C949701B0
:100070000C9497010C9497010C9497010C949701A0
:100080000C9497010C9497010C9497010C94970190
:100090000C9499010C9497010C9497010C9497017E
:1000A0000C9497010C9497010C949701020502059A
:1000B0002E052E05A306A306A306A30696052F0666
:1000C000400640065C1B831B7B1C831B7B1CCF1BD9
:1000D000F21B7B1C491C581C165C1E001F002000D4
:1000E00021002200230024002500260027002D00E7
:1000F0002E0000002A0049002B0014001A000800FE
:10010000150017001C0018000C00120013002F002F
:100110003000000031004C003900040016000700D8
:1001200009000A000B000D000E000F003300340020
:100130000000510028004B00E10000001D001B00E2
:1001400006001900050011001000360037003800C5
:10015000E5004F0052004E00E000E300E200000026
:10016000000000002C00000000000000E600E40099
:10017000015150000000000035003A003B003C00F7
:100180003D003E003F00400041004200430044006B
:100190004500000068006900295C010001000100C1
:1001A0000100010001000100010001000100010047
:1001B000010000000100C35C1F5C010001000100A0
:1001C0000100010001000100010001000100010027
:1001D0000000C75C005CC45C01000000010001007D
:1001E0000100010001000100285CCB5CCA5C010039
:1001F0000100C85CC65C01000100010001000000B4
:1002000000000000010000000000000001000100EB
:100210000100C95C0000000012034C0046004B00C6
:10022000360035005F0048005300000018034C0002
:1002300046004B006500790062006F0061007200AB
:100240006400730000000403090409022200010194
:1002500000A0FA09040000010301010009211101B5
:10026000000122400007058103080001120100027D
:1002700000000008EDFE64600100010200010501BC
:100280000906A101050719E029E7150025019508D0
:10029000750181029501750881010507190029FF83
:1002A000150026FF0095067508810005081901292B
:1002B00005950575019102950175039101C0112401
:1002C0001FBECFEFDAE0DEBFCDBF04B603FE18C01D
:1002D0008091240290912502A0912602B0912702DC
:1002E0008730904BA740B04B59F4109224021092E3
:1002F00025021092260210922702E0E0F8E3099509
:1003000011E0A0E0B1E0ECE0FAE302C005900D924C
:10031000A632B107D9F722E0A6E2B1E001C01D92F2
:10032000A432B207E1F70E9458120C94041D0C94F9
:1003300000001F920F920FB60F9211242F933F933C
:100340004F935F938F939F93EF93FF938091B900A7
:10035000887F883239F180F4803109F4A6C030F406
:10036000882309F4A6C08830E9F0AAC08831B9F022
:10037000803209F487C0A4C08034B1F138F48033EE
:1003800009F480C0883309F47DC09AC08035E1F15A
:10039000883509F45CC0883409F092C073C083E0EA
:1003A0008093F0012091F3013091F4018091FB01E1
:1003B0009091FC01281739070CF05AC02091F501E3
:1003C0003091F6018091F3019091F401AC014F5FFF
:1003D0005F4F5093F4014093F301F901E80FF91FC7
:1003E00080818093BB002EC084E08093F0018091D7
:1003F000F7019091F80101972091F9013091FA01EC
:1004000028173907FCF419C08091F9019091FA017D
:100410009C012F5F3F4F3093FA012093F9014091E7
:10042000BB00FC01E452FE4F40838091F7019091A4
:10043000F8010197281739072CF488EF8093F10110
:1004400085EC3CC088EF8093F10185E837C080914E
:10045000F9019091FA019C012F5F3F4F3093FA010F
:100460002093F9012091BB00FC01E452FE4F208350
:100470008091F201882311F08FEF0BC01092F001F0
:100480008FEF10C08091F201882339F08091B9007C
:10049000887F8093F10185EA11C01092F00180916C
:1004A000B900887F8093F10108C082E08093F00159
:1004B00007C01092F1011092F00185E98093BC0011
:1004C000FF91EF919F918F915F914F913F912F916C
:1004D0000F900FBE0F901F9018950F931F93CF93FF
:1004E000DF93EC018B01C1158CE5D80711F40E9454
:1004F000D602B801CE01DF91CF911F910F910C94DC
:10050000830281E0089581E0089508950C948502A6
:100510001F93CF93DF9300D000D01F92CDB7DEB7EB
:1005200049835A836B833091290189819A813111E2
:1005300014C0662359F0222349F00E94D408182FD2
:10054000682F89819A810E947D0803C00E94A808B3
:10055000182F69817A81812F04C00E94D408698193
:100560007A810F900F900F900F900F90DF91CF91A5
:100570001F910C94D80FFC01262F4081518162817C
:10058000738184810C94880281E00895CF93DF9376
:10059000EC0160E00E94BB02BE01DF91CF910C94A0
:1005A00086020C9409110C94051108950E942707E6
:1005B0000E94D5022FEF84E39CE0215080409040C0
:1005C000E1F700C000000C9426160F931F93CF9301
:1005D000DF938C0161E00E94BB02EC01B8010E9434
:1005E0006D028823F1F1B801CE010E9451148823D5
:1005F000C1F1B801CE010E946512882391F1B801C2
:10060000CE010E94AD13882361F1F8018281882315
:1006100009F1CB358DE5D807C1F050F4C115FCE5E3
:10062000DF0781F0CF3DDC45A9F40E94050E19C01B
:10063000CC35EDE5DE0761F0CD35DD4559F40E949E
:100640004E0D08C00E94D6020CC00E94570D02C079
:100650000E945A0DC801DF91CF911F910F910C9408
:10066000810280E0DF91CF911F910F9108950E9448
:100670005A150C9450030E9453030C94601508956E
:100680000C943F0381E008950C9442030895CF93A6
:10069000C82F0E9440038C2F0E944403CF910895DD
:1006A00080E00C9447030E94AD140C9447030E9411
:1006B000AD1490912801891721F0809328010C94A2
:1006C00047030895CF93DF93CDB7DEB72B970FB6CF
:1006D000F894DEBF0FBECDBF4F83588769877A87F6
:1006E0008B8761110E949A0C9E012F5F3F4F86E01D
:1006F000F90111928A95E9F785E0FE013796D90153
:1007000001900D928A95E1F789819A814C815D81F2
:10071000452B31F09F3F31F491E08F3F19F403C036
:1007200091E001C090E090FF09C049815A816B813E
:100730007C818D819E810E94BB0B05C0C9010E94F6
:10074000C4028111F2CF2B960FB6F894DEBF0FBE14
:10075000CDBFDF91CF910895FC01808191810E94EE
:1007600016090895CF93882309F482C0C82F8238D0
:10077000C1F40E94AD1481FD7BC069E38091020148
:10078000909103010E9432150E94BC0C2FEF81EE64
:1007900094E0215080409040E1F700C0000069E300
:1007A00019C08338F1F40E94AD1480FD61C063E587
:1007B00080910201909103010E9432150E94BC0CAD
:1007C0002FEF81EE94E0215080409040E1F700C08F
:1007D000000063E580910201909103010E943415AD
:1007E00044C08438C1F40E94AD1482FD41C067E466
:1007F00080910201909103010E9432150E94BC0C6D
:100800002FEF81EE94E0215080409040E1F700C04E
:10081000000067E4DFCF8CEF8C0F813AD0F46C2FAF
:1008200080910201909103010E94FC14882349F0F9
:100830006C2F80910201909103010E9434150E9457
:10084000BC0C6C2F80910201909103010E94321523
:100850000CC080E28C0F883058F4C77081E001C072
:10086000880FCA95EAF70E947D0CCF910C94BC0CBE
:10087000CF910895882309F45BC0682F823879F4FA
:100880000E94AD1481FF54C069E3809102019091F0
:1008900003010E9432150E94BC0C69E310C083382A
:1008A000B1F40E94AD1480FF43C063E58091020162
:1008B000909103010E9432150E94BC0C63E5809167
:1008C0000201909103010E9434150C94BC0C8438F1
:1008D00079F40E94AD1482FF2BC067E4809102017D
:1008E000909103010E9432150E94BC0C67E4E7CF8F
:1008F0008CEF860F813A18F380E2860F883048F437
:10090000677081E001C0880F6A95EAF70E94830C46
:10091000DCCF8BE5860F833020F480E090E00C94F0
:10092000C414685A673120F480E090E00C94DA1423
:1009300008951F93CF93DF93182FEB010E94B2030A
:10094000209741F08FE99FE00197F1F700C0000088
:100950002197F6CF812FDF91CF911F910C943A040C
:10096000893319F060E070E002C060E570E00C943B
:100970009904882321F00E947D0C0C94BC0C0895EE
:10098000882321F00E94830C0C94BC0C0895CF9214
:10099000DF92EF92FF920F931F93CF93DF937C012F
:1009A000D62FC72FFC011281058102950F700E947E
:1009B000730C8823B9F01123A9F08C2F807F803429
:1009C00021F080E28D0F883068F08091FE0182FD79
:1009D00009C082E00E941C0D0E94730C91E0D82E89
:1009E000D92601C0D12CCC2EC2948FE0C8228C2DE8
:1009F00090E08C30910508F0A6C1FC01EA5AFF4F47
:100A00000C94AF1C8C2F807FCF70882311F0C2957F
:100A1000C07F112399F0CC2309F481C180E28D0FAE
:100A2000883010F0D11104C08C2F0E947D0C03C0BF
:100A30008C2F0E948D0C0E94BC0C71C18D2F0E94C6
:100A40003A04CC2309F47FC180E28D0F883038F15D
:100A5000DD2329F18C2F0E94930C24C08C2F807FE2
:100A6000CF70803211F0C295C07FDD2319F0D130F4
:100A7000A1F13DC08091FE0182FF17C0112349F012
:100A8000CC2329F08C2F0E947D0C0E94BC0C80E0AE
:100A900047C180E00E943A04CC2309F454C18C2F52
:100AA0000E94830C0E94BC0C4EC1112371F00023E4
:100AB00041F0013031F40E949D0C8C2B0E94A50C5A
:100AC00042C10E949D0C8C2B1DC0002319F00130E7
:100AD00009F439C10E94B20C25C0112321F006305F
:100AE00008F031C10EC0053008F02DC11BC0112324
:100AF00061F0002331F0F701858180FF10C18F7014
:100B000085838C2F0E94B9041EC1002359F0D9336C
:100B100009F016C1FFEF07EE13E0F150004010405E
:100B2000E1F70CC18C2F0E94C0040DC18C2F837083
:100B300009F047C011110BC12D2F22952695277062
:100B4000220F220F6D2F6F70862F90E0A0E0B0E093
:100B5000022E04C0880F991FAA1FBB1F0A94D2F748
:100B6000D4FF10C04FE050E060E070E004C0440FDC
:100B7000551F661F771F2A95D2F7409550956095AF
:100B8000709503C040E050E0BA01C695C695C370A9
:100B90008A019B01082B192B2A2B3B2BC901B80179
:100BA000C23049F058F4C13019F00E949307CFC009
:100BB0000E948107CCC00E94A507C9C00E947F0780
:100BC000C6C0112319F08C2F817001C0869588232F
:100BD00009F4BDC02D2F229526952770220F220FD4
:100BE0006D2F6F70862F90E0A0E0B0E0022E04C061
:100BF000880F991FAA1FBB1F0A94D2F7D4FF10C0F9
:100C00004FE050E060E070E004C0440F551F661FE5
:100C1000771F2A95D2F7409550956095709503C03F
:100C200040E050E0BA01C695C695C3708A019B01A9
:100C3000082B192B2A2B3B2BC901B801C23049F0D4
:100C400058F4C13019F00E94580881C00E9446082B
:100C50007EC00E946A087BC00E94B90778C0CF702E
:100C6000112339F08C2F0E94DF078D2F0E94B904C9
:100C70006EC08D2F0E94C0048C2F0E94000867C098
:100C8000D23F21F128F4D03F41F0D13FC1F043C021
:100C9000D33F19F1D43F79F03EC0112341F0053024
:100CA00008F051C08C2F8F710E9425084CC006306F
:100CB00008F049C0F7CF8091FE0182FF18C01123D0
:100CC00039F08C2F8F710E94DF073DC01123C9F3CB
:100CD0008C2F8F710E94000836C0112329F08C2FB1
:100CE0008F710E94CA072FC00E94C5072CC0112314
:100CF00049F0CF718C2F0E94DF0763E08C2F0E9498
:100D0000010D21C081E00E941C0D0230E0F082E064
:100D10000E941C0D18C0112331F0002391F28D2F79
:100D20000E94B20310C0002399F2D93349F41FEF97
:100D300027EE33E0115020403040E1F700C00000C2
:100D40008D2F0E943A0488EF8C0D843020F40E948D
:100D5000AD140E944703DD20C9F00E946F0C80FD96
:100D600015C0F70112820E94690C0E94DF07C701BB
:100D70000E94E7060E94690CDF91CF911F910F91AD
:100D8000FF90EF90DF90CF900C940008DF91CF910F
:100D90001F910F91FF90EF90DF90CF9008950F93E8
:100DA0001F93CF93DF93EC01688179818A810E9440
:100DB00021098C010E947C080E946D07B801CE01B8
:100DC0000E94C704DF91CF911F910F910895CF9397
:100DD000DF93EC01988189812B813C81232B31F0B9
:100DE0008F3F31F481E09F3F19F403C081E001C0DF
:100DF00080E080FD1DC0CE010E94E502811110C07F
:100E00000E94730C8823A1F08A81882389F0809145
:100E1000FE0182FD0DC082E0DF91CF910C941C0D8C
:100E2000CE010E94CF06CE01DF91CF910C94C60275
:100E3000DF91CF9108950E949A0C0C94BC0C809184
:100E40000201909103010E9436150C941B070E9429
:100E50008A0C0C941F0792959F70963079F010F4CD
:100E6000925001C09A50923068F4803F69F018F4B3
:100E7000883E40F409C0843F29F406C0883E20F033
:100E8000813F11F080E0089581E00895FC018081A8
:100E900091810E9416090E942B070895CF93DF933A
:100EA00000D000D01F92CDB7DEB70F900F900F90FB
:100EB0000F900F90DF91CF910895CF93DF9300D0E3
:100EC00000D000D0CDB7DEB726960FB6F894DEBFBF
:100ED0000FBECDBFDF91CF910895089508950C9472
:100EE0006E070C946F070E94710760936001709306
:100EF000610180936201909363010C941B070C9431
:100F000073070F931F93009160011091610120916D
:100F1000620130916301602B712B822B932B1F9107
:100F20000F910C9473070F931F9300916001109120
:100F3000610120916201309163016023712382235A
:100F400093231F910F910C9473070F931F9300919C
:100F5000600110916101209162013091630160276D
:100F60007127822793271F910F910C9473070C947C
:100F70006E070E94B70760935C0170935D018093D8
:100F80005E0190935F010C941B0760E070E0CB0161
:100F90000C94B9070F931F9341E050E060E070E0BC
:100FA0008A019B0104C0000F111F221F331F8A9565
:100FB000D2F7C901B8011F910F910C94B9070F9393
:100FC0001F9341E050E060E070E004C0440F551F03
:100FD000661F771F8A95D2F780915C0190915D0121
:100FE000A0915E01B0915F018A019B01082B192B32
:100FF0002A2B3B2BC901B8011F910F910C94B90703
:101000000F931F9341E050E060E070E004C0440F94
:10101000551F661F771F8A95D2F7409550956095AA
:10102000709580915C0190915D01A0915E01B091FD
:101030005F018A019B01082319232A233B23C9014D
:10104000B8011F910F910C94B9070F931F9341E0C2
:1010500050E060E070E004C0440F551F661F771F2A
:101060008A95D2F780915C0190915D01A0915E011B
:10107000B0915F018A019B01082719272A273B2786
:10108000C901B8011F910F910C94B9070F931F93D9
:1010900000915C0110915D0120915E0130915F0132
:1010A000602B712B822B932B1F910F910C94B907FE
:1010B0000F931F9300915C0110915D0120915E01DF
:1010C00030915F0160237123822393231F910F913D
:1010D0000C94B9070F931F9300915C0110915D016F
:1010E00020915E0130915F0160277127822793274D
:1010F0001F910F910C94B907089520E1929F800DE4
:101100001124E82FE695E695E695877051E001C039
:10111000550F8A95EAF785E0E89FF0011124E65D16
:10112000FE4F20E030E070E04081CB01022E02C093
:10113000969587950A94E2F7817081958427852397
:10114000842781932F5F3F4F2530310569F708953C
:1011500020E1929F800D1124682F66956695669513
:10116000982F977085E0689FB001112440E050E00F
:1011700080E0FB01E40FF51FE65DFE4F208130E0CB
:10118000092E02C0369527950A94E2F7217033277D
:10119000042E01C0220F0A94EAF7822B4F5F5F4FA3
:1011A0004530510531F70895BF92CF92DF92EF920B
:1011B000FF920F931F93CF93DF938C01C0905C013C
:1011C000D0905D01E0905E01F0905F018091600140
:1011D00090916101A0916201B0916301C82AD92A5E
:1011E000EA2AFB2ACFE1D0E0D701C6010C2E04C0C9
:1011F000B695A795979587950A94D2F780FD04C078
:10120000219790F7B12C07C0BC2EB8018C2F0E94FB
:10121000ED0F0197A9F38B2DDF91CF911F910F91C6
:10122000FF90EF90DF90CF90BF900895CF93DF9322
:10123000EC010E94D408BE010E94ED0FDF91CF9116
:1012400008951F93CF93DF93EB0190912901992388
:1012500021F0CB010E94160913C0882349F0CB016D
:101260000E94D408182F682FCE010E947D0804C068
:10127000CB010E94A808182FBE01812F0E94ED0FFC
:10128000DF91CF911F9108951F93CF93DF93C0916A
:10129000640116E080916501C81799F0D0E01C9FA9
:1012A000F0011D9FF00D1124EA59FE4F408151813C
:1012B00062817381848195810E945D072196C77048
:1012C000E9CFDF91CF911F91089540919601509100
:1012D0009701609198017091990180919A01909184
:1012E0009B010C945D07EF92FF920F931F93CF9396
:1012F000DF9380919B0182958F7009F065C080918A
:101300009801882309F460C080916401F090650120
:1013100010919601009197016091990170919A0145
:1013200091E01F3F09F090E0C0910001D0910101D0
:10133000292F96E0E92E8F1509F446C06115710535
:1013400021F00F3F21F030E003C031E001C0322F27
:1013500090E030FD36C0E89EF001E99EF00D1124CA
:10136000DF01AA59BE4F11963C911197301329C045
:101370003C91311326C012963C911297311121C035
:1013800013964D915C911497461B570B4C175D07B4
:10139000C0F480919B018F70806180939B01E5591F
:1013A000FE4F80818F708061808386E991E00E948A
:1013B000E706DF91CF911F910F91FF90EF900C9472
:1013C000440901968770B7CFDF91CF911F910F919C
:1013D000FF90EF9008959F92AF92BF92CF92DF92CD
:1013E000EF92FF920F931F93CF93DF93CDB7DEB7AA
:1013F00061970FB6F894DEBF0FBECDBF8C0185E0BC
:10140000F801DE011D9601900D928A95E1F7D80151
:101410001296EC9090919601E0919701209199019C
:1014200030919A012115310531F0EF3F31F481E01F
:101430009F3F19F403C081E001C080E0B82FB17074
:101440009B2E80FD47C1D8014C9111965C9111975C
:101450001396AD90BC90149786E9C82E81E0D82EE3
:10146000F0909801B501621B730B2091000130913F
:101470000101FF2009F4D9C080919B016217730715
:1014800008F095C0282F207F09F052C05E1313C0CA
:10149000491311C0FE2CE1100EC08F708061809343
:1014A0009B010E946509C6010E94E70680919B018D
:1014B000F80185834DC1AB2831F05F3F31F481E005
:1014C0004F3F19F403C081E001C080E080FD03C0FC
:1014D00081E08E2502C080E090E0F82FF170FF2EB1
:1014E00080FF1CC0809164012091650136E0821765
:1014F00009F40BC190E0389FF001399FF00D1124E1
:10150000EA59FE4F6181561306C06081461303C03D
:101510006281E61203C001968770E9CFFE2CEE20AF
:1015200009F416C180919B01816080939B0154C096
:101530005E1306C0491304C0E11002C0F80199C04F
:10154000C8010E944607882361F1EE2051F12091E5
:101550009B01822F82958F7090E0029774F08091AA
:1015600096019091970198878F831986BB86AA86EA
:101570002C87CE0107960E94E70686E0F801A6E9CF
:10158000B1E001900D928A95E1F70E9473090E94E3
:1015900065090AC05E1711F1C8010E944607811152
:1015A0002CC0C8010E94E706FF24F394D1C0282F65
:1015B000207F81F77A2DB98AA88A6E2D89890E94A9
:1015C0004E0786E991E00E94E70686E0D6011D926B
:1015D0008A95E9F70E946509F12CBAC04913DCCF5E
:1015E000E110DACFF8018583C8010E94E70686E0A2
:1015F000D6011D928A95E9F7ABC0EE2091F22091B9
:101600009B01822F82958F7090E002970CF4B5CFEA
:1016100080919601909197019A8389831B82BD8264
:10162000AC822E83CE010196A6CF6217730708F015
:1016300044C0FE2CEE2009F4B4CF5E1330C0491331
:101640002EC020919B0120FD21C0822F82958F709A
:10165000482F50E041155105C9F0F80125834F305E
:10166000510541F08F5F982F9295907F822F8F7058
:10167000892B8583C8010E94E70686E0F801A6E968
:10168000B1E001900D928A95E1F73CC086E0F80147
:10169000A6E9B1E001900D928A95E1F759C0C80121
:1016A0000E944607811169CF80919B0181608093E0
:1016B0009B01C8010E94E7064BC07A2DB98AA88A0F
:1016C0006E2D89890E944E0786E0D6011D928A956B
:1016D000E9F718C0EE2009F464CFC8010E9446075C
:1016E000F82E882309F45DCF86E0F801A6E9B1E081
:1016F00001900D928A95E1F786E991E00E94AC0392
:101700000E9473090E94650923C04D875E878D85FD
:101710009E850E941609292F22952F70223028F4C9
:101720009F7039F0811105C00BC0243028F49F70E0
:1017300049F4805E883020F0C8010E94E7069F2CA3
:10174000F92C06C0D80115969C91907F91F7F8CF9F
:101750008F2D61960FB6F894DEBF0FBECDBFDF911F
:10176000CF911F910F91FF90EF90DF90CF90BF909E
:10177000AF909F9008951F93CF93DF93CDB7DEB7BF
:101780002C970FB6F894DEBF0FBECDBF4F8358879E
:1017900069877A878B879C87CE0107960E94EB0921
:1017A0008823D1F09F8188852A853B85232B31F0C2
:1017B0008F3F31F481E09F3F19F403C081E001C005
:1017C00080E080FD47C04F81588569857A858B858B
:1017D0009C850E945D073EC086E0FE013796DE01D3
:1017E000119601900D928A95E1F7FF81E8856A854F
:1017F0007B856115710531F0EF3F31F481E0FF3FEA
:1018000019F403C081E001C080E080FD23C0209175
:10181000650130E0C9010196877099274091640104
:1018200050E084179507F1F1F983EA837D836C8397
:1018300096E0929FD001939FB00D1124AA59BE4FFC
:10184000FE01319601900D929A95E1F78093650122
:101850000E94440916E08091640190916501891706
:1018600071F1189FC00111248A599E4F0E94EB0903
:10187000882329F1E09164011E9FF0011124EA59A7
:10188000FE4F4081518162817381848195810E94E4
:101890005D078091640190E001968770992780939D
:1018A0006401D9CF0E94270710926501109264014C
:1018B000E6E9F1E086E0DF011D928A95E9F72C96D2
:1018C0000FB6F894DEBF0FBECDBFDF91CF911F9151
:1018D00008958091A40185958595859508958091B9
:1018E000A401877008959091A401977081E009F494
:1018F00080E008958091AF0108959091AF01892B08
:101900008093AF01089580959091AF0189238093D2
:10191000AF0108951092AF0108959091AE01892B07
:101920008093AE01089580959091AE0189238093B4
:10193000AE0108951092AE0108958091A501089519
:1019400008950C94A00C0C94A10C9091FE0192FDB2
:1019500008C09091A501981721F08093A5010C94DF
:10196000A30C08958091A501882329F01092A50168
:1019700080E00C94A30C0895CF93DF93E0910201D3
:10198000F09103018091AF018083E0910201F09119
:10199000030190818091AE01892B80838091A50104
:1019A000882381F0E0910201F09103019081892B5D
:1019B000808380910201909103010E94F0148111B3
:1019C0000E94B20CC0910201D091030148E050E0A6
:1019D0006CE971E0CE010E94B51C892B69F088E0AA
:1019E000FE01ACE9B1E001900D928A95E1F7CE01DC
:1019F000DF91CF910C94B914DF91CF9108950C949D
:101A0000A00C9091FE0192FD10C098E0899F90017A
:101A10001124262B2093A4010E94DF078091A401AA
:101A20008595859585950C94FF0C0C94DF07109295
:101A3000A40180E00C94FF0C2091A40180958223E6
:101A40008093A401982F977099F430E0482F082EC6
:101A5000000C550B2417350759F09091FE0192FDAB
:101A600007C08595859585950E9400080C94170DF3
:101A700008959091FE0192FB222720F9281769F022
:101A800080FB92F99093FE018091FD019091FE01FF
:101A90000E94810D82E00C941C0D08958091FE013E
:101AA00082FB882780F991E089270C94390D81E029
:101AB0000C94390D80E00C94390D80E090E00E9488
:101AC000CA1C21E0893E9E4F09F020E0822F089534
:101AD00082E090E00C94C21C83E090E00C94C21C65
:101AE000CF9384E090E00E94C21CC82F82E290E075
:101AF0000E94C21C2C2F30E0A901582BCA01CF91A3
:101B00000895CF93C92F682F84E090E00E94D01CE5
:101B10006C2F82E290E0CF910C94D01CAB01BC0101
:101B20008FE090E00C94E21CAB01BC0183E190E0FB
:101B30000C94E21C60E070E0CB010C94940D60E02A
:101B400070E0CB010E948E0D0C949A0D69EE7EEF31
:101B500080E090E00E94EE1C60E082E090E00E9455
:101B6000D01C60E083E090E00E94D01C10926001E5
:101B700010926101109262011092630160E084E0B2
:101B800090E00E94D01C60E082E290E00E94D01CB5
:101B900060E085E090E00E94D01C60E086E090E08C
:101BA0000E94D01C6FEF87E090E00E94D01C40E0C4
:101BB00050E0BA0188E090E00E94E21C60E08DE015
:101BC00090E00E94D01C40E050E0BA0188E190E033
:101BD0000E94E21C60E087E190E00E94D01C40E09F
:101BE00050E0BA018CE190E00E94E21C60E070E0FD
:101BF00080E290E00E94EE1C40E050E0BA0188E1F3
:101C000090E00E94E21C0C949F0D0C94A60D682F8E
:101C10008EE090E00C94D01C0E94E5156093BE010C
:101C20007093BF018093C0019093C1016093BA018A
:101C30007093BB018093BC019093BD01089585B75B
:101C4000806885BF85B7806885BF089581E0089565
:101C50000C94260E08950C942A0E0C942A0E0C94C3
:101C60002D0E0C942A0E0C94310E0C942A0E0E9408
:101C70001F0E89EC90E10E94A3140E94350E0C9473
:101C8000330E0E942B0E0C942A0E0E94CC100C9442
:101C900046030E94D0150E94B1110E94450E0C947B
:101CA0002F0E5F926F927F928F929F92AF92BF9210
:101CB000CF92DF92EF92FF920F931F93CF93DF9318
:101CC000CDB7DEB72A970FB6F894DEBF0FBECDBFF3
:101CD0000E94C611C82E81110E940C0E30EB832E7B
:101CE00031E0932E00E010E0502E802F0E94F01083
:101CF0005C01F401619071904F01682679266114AE
:101D00007104B1F40F5F1F4F0530110569F78FEFB4
:101D100089838A831B820E94D9158160782F9D83D5
:101D20008C8349815A816B818D810E9462033AC004
:101D30008091C20181FD0E94F910D12CEE24E39420
:101D4000F12CC3018E219F21892B29F10E94280E9D
:101D50008823A9F0DE825F82AE20BF2081E0AB281D
:101D600009F480E088870E94D9158160782F9A87CE
:101D700089874E815F8168858A850E946203000F92
:101D8000111FF801E055FE4F80819181E826F92668
:101D9000F182E08207C0D394EE0CFF1CF0E1DF1269
:101DA000D0CFB0CF81E0C11001C080E02A960FB63D
:101DB000F894DEBF0FBECDBFDF91CF911F910F9181
:101DC000FF90EF90DF90CF90BF90AF909F908F905B
:101DD0007F906F905F9008950E94510E0C9457036E
:101DE000CF93DF930E94F20FEC01811523E5920758
:101DF000A0F5811532E5930708F09EC0811540E2F9
:101E00009407C0F4811551E0950708F0CDC0853ADC
:101E1000910550F48430910508F0C6C0019709F08F
:101E2000C0C081E090E0C1C0805E9109089708F4CD
:101E3000BBC0B7C0C11581E5D80708F077C0C11590
:101E400020E5D20708F051C0C11530E4D30708F4EB
:101E5000A8C0DF70CE01906AA8C0811546E594073E
:101E600000F5811555E5950708F081C0C11584E599
:101E7000D80708F076C0CE018370992721E030E0C2
:101E800002C0220F331F8A95E2F79C2F96959695F4
:101E900040E2949FE0011124C22BD32BCE019A681B
:101EA00084C081152AE5920780F4811539E59307EE
:101EB00008F066C0811548E5940708F472C0D82F71
:101EC000CC27CE01806F906A70C0905681159042E9
:101ED00008F067C08D2F8F710E948610DD27D062B9
:101EE0008F71AE01582BCA0160C0CE0174E0969587
:101EF00087957A95E1F7282F23703C2F337081E086
:101F000090E002C0880F991F3A95E2F79C68AC01F7
:101F1000522B9A019C2F9F709695969550E2959F13
:101F2000E0011124C9018C2B9D2B3FC0DC2FCC2755
:101F3000CE01816F906A39C08370992721E030E02B
:101F400002C0220F331F8A95E2F79C2F9695969533
:101F500080E2989FE0011124C22BD32BCE019C6814
:101F600024C0DC2FCC27CE01846F906A1EC00E9453
:101F700086108F7190E0D82FCC27CE01906215C0CB
:101F80008F700E94861094E0D695C7959A95E1F7D8
:101F9000CF70D0E0DC2FCC27D0699E01282BC9015F
:101FA00004C080E090E001C0CE01DF91CF910895A0
:101FB000E72FF0E095E0899FE00DF11D112484E00A
:101FC000EE0FFF1F8A95E1F7E60FF11DEE0FFF1FE1
:101FD000E852FF4F8591949108950E94D80F0E9476
:101FE000F00E08958238910569F1B0F481339105BE
:101FF00009F46DC048F48932910509F463C08A324E
:10200000910509F469C008958533910509F455C017
:1020100089339105B9F00895833E910569F138F44B
:10202000803E9105B1F0823E910509F10895863E0A
:102030009105A9F1873E9105B9F1843E910509F01A
:1020400064C023C02091FD0120FD4FC021FD4DC083
:1020500008958091FD0180FD44C08091FE0180FFC4
:1020600044C08091FD0184FD42C083EE4DC080914B
:10207000FD0182FF38C0F5CF8091FD0182FD33C0A4
:102080008091FE0180FD31C0ECCF8091FE0181FF87
:1020900032C08091FD0184FD2AC087EE35C0809159
:1020A000FD0183FF26C0F5CF8091FD0183FD21C096
:1020B0008091FE0181FD1FC0ECCF8091FD0185FD67
:1020C0001CC01DC08091FD0185FD19C016C0809106
:1020D000FD0186FD16C017C08091FD0186FD13C06D
:1020E00010C089E311C082EE0FC080EE0DC080E009
:1020F0000BC086EE09C084EE07C089E205C085E307
:1021000003C08AE201C081E390E008959091FD014F
:1021100092FF0DC0282F2871283019F4877F846022
:1021200006C0282F2471243011F48B7F886093FF20
:102130000DC0282F2871283119F4877E846106C0CC
:10214000282F2471243111F48B7E88612091FE01A7
:1021500020FF0DC0382F3871383019F4877F816027
:1021600006C0382F3171313011F48E7F886021FF25
:102170000DC0282F2871283119F4877E816106C08F
:10218000282F2171213111F48E7E886194FD877E84
:10219000089580E0089508950E945D0D811102C0A8
:1021A0000E94050E0E94680D8093C2010E94700D6E
:1021B0009093FE018093FD010E94CB100E946C0D54
:1021C000682F70E080E090E00E947F0760915C01E2
:1021D00070915D0180915E0190915F010C94B70751
:1021E000E82FF0E0EE0FFF1FE75FFD4F8081918148
:1021F0000895089580EA8A95F1F7089500C008953A
:102200000C94FA1008950C9402110C9403110C9480
:1022100002110C940711F894E82FE295EF70F0E0AA
:1022200031A1282F2F7081E090E001C0880F2A95FE
:10223000EAF7982F9095932391A392A1892B82A3DB
:10224000789408950F931F93CF93DF93C1E2D1E069
:1022500089918F3F11F00E940B1181E0C632D8079F
:10226000B9F7C1E1D1E001E211E089918F3F11F0AE
:102270000E940B110C171D07C1F7DF91CF911F9121
:102280000F910895BF92CF92DF92EF92FF920F933A
:102290001F93CF93DF938C01C62FD0E0CE018F5DCB
:1022A0009E4F6C01FC0190819F3F09F450C0B62EF7
:1022B000F894E92FE295EF70F0E081A19F7021E0A2
:1022C00030E001C0220F9A95EAF7822B81A382A108
:1022D0002095282322A378940E94FE10E1E1F1E0EA
:1022E00041E251E021E030E0E12CF12C61916F3FBF
:1022F00089F0A62FA295AF70B0E090968C9190E0F7
:102300006F7002C0959587956A95E2F780FD02C0CF
:10231000C90102C080E090E0E82AF92A220F331FA9
:102320004E175F0719F7F60180818F3F11F00E9469
:102330000B1161E0E114F10409F460E08B2D0E94BF
:102340000011CC0FDD1FC00FD11FF982E882DF9191
:10235000CF911F910F91FF90EF90DF90CF90BF90A2
:1023600008950E9422118AE0E9E0F2E0DF01982F4F
:102370001D929A95E9F7EFEFF1E0DF011D928A9542
:10238000E9F785E00E9411120C94D102FF920F939D
:102390001F93CF93DF93CDB7DEB72A970FB6F8948C
:1023A000DEBF0FBECDBF8E010F5F1F4F8AE0F80169
:1023B00011928A95E9F7F12C6F2DC8010E94421104
:1023C000F394F5E0FF12F8CF4AE050E0B8018FEF48
:1023D00091E00E94B51CFF24F394009709F4F12CBE
:1023E000892B41F08AE0F801AFEFB1E001900D9246
:1023F0008A95E1F72F2D45E069E072E08FEF91E0DB
:102400000E9412120E94D3028F2D2A960FB6F894C2
:10241000DEBF0FBECDBFDF91CF911F910F91FF9017
:1024200008950895FF920F931F93CF93DF93F82E93
:10243000092F162FD72FC42F222349F081E0809334
:10244000C5010E94D9159093C4018093C301809166
:10245000C5018823D9F08091C3019091C4010E94E5
:10246000F115059798F0EF2DF02FA12FBD2F80E0EB
:1024700090E04C2F50E08417950734F4219131916E
:102480002D933D930196F7CF1092C501DF91CF9127
:102490001F910F91FF9008950E9488170E94490E86
:1024A0000C9494170E9498170E94EC0E0C94B2178B
:1024B0000E9477150E946F170E94370E0E944C12DF
:1024C0000E9452120E94410EFBCFCF93DF93EC018A
:1024D000FB018281882309F43CC1C430FDE5DF079C
:1024E00060F4CB3F9CE5D90788F49E0122503C451F
:1024F0002431310508F02EC109C0C236EDE5DE07F2
:1025000029F0C63AFDE5DF0709F024C10E94700DED
:102510009093FE018093FD01C1318CE5D80709F449
:10252000C6C008F042C0C930ECE5DE0709F49BC024
:1025300000F5C5308CE5D80709F485C078F4C330C0
:10254000ECE5DE0709F478C008F07AC0C230DC455B
:1025500009F0F5C08091FD018160EFC0C7309CE5B6
:10256000D90709F478C008F07AC08091FD01806134
:10257000E4C0CD30FCE5DF0709F487C058F4CB3068
:102580009CE5D90709F479C008F07BC08091FD0172
:1025900088606FC0CF30FCE5DF0709F480C008F029
:1025A00082C08091FD01877FC8C0CE3F9CE5D907DE
:1025B00009F471C000F5C531FCE5DF0709F485C0F9
:1025C00068F4C3319CE5D90709F475C008F095C0DB
:1025D0000E9427078091FD018F77AFC0CC3FFCE5BB
:1025E000DF07A9F108F054C0CB3FDC4509F0A7C0D4
:1025F0008091FE0140C0C230EDE5DE0709F489C0DC
:1026000058F4C1158DE5D80709F45AC008F069C01F
:102610008091FE0182602FC0C236EDE5DE0709F42D
:102620007CC0C63AFDE5DF0709F481C0C330DD4553
:1026300009F085C080E06EC08091FD0182607DC0A0
:102640008091FD0116C08091FD01886076C0809167
:10265000FE0182604FC08091FD0180626EC080915A
:10266000FD0180646AC00E9427078091FD01806897
:1026700064C0846062C081603DC08091FD018E7F36
:102680005CC08091FD018D7F58C08091FD0116C016
:102690008091FE0118C08091FE018D7F2BC080913A
:1026A000FD018F7E4AC08091FD018F7D46C08091E3
:1026B000FD018F7B42C08091FD01877F8B7F3DC0F4
:1026C0008091FE018D7F8E7F15C08091FD0182FB80
:1026D000222720F991E0922790FB82F990FB83F961
:1026E0002CC08091FE01982F909591708E7F892B40
:1026F00090FB81F98093FE0122C00E942707809100
:10270000FD0187FB222720F991E0922790FB87F9B2
:1027100014C081E00E94070E12C08091FD0184FB6D
:10272000222720F991E0922790FB84F906C080913E
:10273000FD01982F909590FB80F98093FD01809189
:10274000FD019091FE010E94810D0E94270780E00B
:1027500001C081E0DF91CF910895CF93DF9386315F
:102760009C4541F5EB010E947A0C982F8A812091BB
:10277000020130910301882379F09A7A81E009F40B
:1027800080E08093C601911102C069E201C065E357
:10279000C9010E9432150AC08091C601811102C090
:1027A00069E201C065E3C9010E9434150E94BC0CB6
:1027B00080E001C081E0DF91CF9108950F931F93D6
:1027C000CF93DF93C42FD22FFC0182818823C9F0DD
:1027D0004093C9010E94D9159093C8018093C70105
:1027E00080E28C0F883008F057C0C77081E001C0CC
:1027F000880FCA95EAF7DF91CF911F910F910C9442
:10280000B9048091C901481330C08091C7019091EB
:10281000C8010E94F115883C910538F510E21D0FA2
:10282000CD17B9F080E28C0F883040F4C77081E09A
:1028300001C0880FCA95EAF70E94C004183028F535
:1028400081E09D2F977001C0880F9A95EAF70E944A
:10285000B904802F0E94B0041830F0F4D77081E0E2
:1028600001C0880FDA95EAF70AC080E28C0F883041
:1028700098F4C77081E001C0880FCA95EAF7DF912C
:10288000CF911F910F910C94C004802FDF91CF91B5
:102890001F910F910C94B004DF91CF911F910F9174
:1028A00008950F939C01CB01243F4CE5340731F18F
:1028B00088F4293DFCE53F07D9F02A3D4CE5340773
:1028C00079F1283D3C45A9F506E221EE41EE68ED9F
:1028D0007CE52BC0263FFCE53F07E1F0A8F0273F51
:1028E0003C4539F507E225EE46EE67EF7CE51DC075
:1028F00007E225EE45EE69ED7CE517C006E221EE24
:1029000040EE64EF7CE511C007E225EE44EE65EF92
:102910007CE50BC006E221EE42EE66EF7CE505C0E9
:1029200008E221E045EE6AED7CE50E94DE1380E0DE
:1029300008C0FC018281882319F01092C90101C0EE
:1029400081E00F91089590932701809326010895C7
:102950009093CF018093CE010895E091CE01F09144
:10296000CF01309721F00190F081E02D099480E0B3
:102970000895E091CE01F091CF01309721F00280CF
:10298000F381E02D099408952091CC013091CD017F
:102990002817390771F09093CD018093CC01E09115
:1029A000CE01F091CF01309721F00680F781E02D24
:1029B000099408952091CA013091CB012817390755
:1029C00071F09093CB018093CA01E091CE01F09118
:1029D000CF01309721F00084F185E02D099408950E
:1029E000FC01329697E080E0915029F0219122235A
:1029F000D9F38F5FF9CF0895662349F0FC01329631
:102A000008962191621729F0E817F907D1F780E0BD
:102A1000089581E008959C01FC0132969FEF80E0CB
:102A20004191461789F09F3F19F4411101C0982F39
:102A30008F5F8630A9F79F3F39F0F901E90FF11D4B
:102A400097FDFA956283089508959C012A5F3F4F90
:102A5000FC014281461301C012820196821793073E
:102A6000B9F708950C940B150C942515029626E0E1
:102A7000FC0111922A95E9F7089508950C943D15EB
:102A800083E08093D0010C943E15811102C081E057
:102A900001C082E08093D0010C943E150C94451542
:102AA00081E08093D0010C943E150C94501508954C
:102AB0000C9457150C9458150C9457150C945715E5
:102AC0000C945715CF930E945E150E94C6110E9468
:102AD0005C15C0E08C2F0E94F010892B29F4CF5F89
:102AE000C530C1F780E001C081E0CF91089508951D
:102AF0001F920F920FB60F9211248F939F93AF9353
:102B0000BF938091D101811113C0809113029091E4
:102B10001402A0911502B09116024196A11DB11D9B
:102B20008093130290931402A0931502B09316029F
:102B3000BF91AF919F918F910F900FBE0F901F90FB
:102B4000189580911B02843031F10E943703109256
:102B5000D10120E488E190E00FB6F894A895809325
:102B600060000FBE2093600083B7817F846083BFC5
:102B700083B7816083BF7894889583B78E7F83BF46
:102B80000FB6F894A89580916000886180936000EA
:102B9000109260000FBE08950E9427070C943B031B
:102BA00082E084BD93E095BD9AEF97BD80936E005F
:102BB00008952FB7F8948091130290911402A09178
:102BC0001502B09116022FBF08952FB7F8946091A7
:102BD00013027091140280911502909116022FBF7A
:102BE00008959C014FB7F8948091130290911402BC
:102BF000A0911502B09116024FBF821B930B08954E
:102C000078941F920F920FB60F9211248F939F9377
:102C1000AF93BF938091130290911402A09115027B
:102C2000B09116020196A11DB11D809313029093DD
:102C30001402A0931502B0931602BF91AF919F9119
:102C40008F910F900FBE0F901F90189581E0809389
:102C5000E00080E28093D8001092C9008FE19EE4EA
:102C60000197F1F700C0000087E090EBDC01809352
:102C7000240290932502A0932602B09327029CE0A1
:102C800088E10FB6F894A895809360000FBE9093EA
:102C90006000FFCF8091DA01089508950895CF93E1
:102CA000DF9321E02093E9002FEF3091E8002150DD
:102CB00035FD06C035ED3A95F1F700002111F5CF4D
:102CC0002091E80025FF14C0EC0140E050E068E0EE
:102CD00070E00E9411188091E8008E778093E800E0
:102CE00088E0FE01A2EDB1E001900D928A95E1F736
:102CF000DF91CF9108950895089580911A0281116E
:102D000009C00E94A2190E94FF198091E20084600C
:102D10008093E200089510921A0208950C945515BC
:102D20006091170281E0611101C080E00C944015B0
:102D300090911B0281E0943009F080E060911702CD
:102D40000C94451542E061EC81E00E941B199091C2
:102D50001B0281E0943009F080E0609117020C942E
:102D60004E1580911D02833009F461C030F481302A
:102D700071F0823009F49AC008958A3009F486C04F
:102D80008B3009F46CC0893009F0A8C020C0809154
:102D90001C02813A09F0A2C08091E800877F8093ED
:102DA000E8008091200290912102892B21F468E0B3
:102DB00082ED91E003C060E080E090E070E00E946E
:102DC0005C188091E8008B778093E80008958091EB
:102DD0001C02813209F082C0809120029091210270
:102DE000892B09F07BC08091E800877F8093E80001
:102DF0008091E80082FD05C080911B028111F8CF0F
:102E00006DC02091F3008091F20090E0922B029728
:102E100031F48091F100813011F0863021F48091FD
:102E2000F1008093DA018091E8008B7753C08091A4
:102E30001C02813A09F052C0809120029091210237
:102E4000892B09F04BC08091E800877F8093E800D0
:102E50008091E80080FFFCCF8091100136C0809106
:102E60001C028132D9F58091200290912102892B98
:102E7000A9F58091E800877F8093E8000E945019AF
:102E800080911E02809310010C94270780911C02F0
:102E9000813221F58091E800877F8093E8000E94CD
:102EA000501980911F028093DB01089580911C02CC
:102EB000813AA1F48091E800877F8093E8008091B7
:102EC000E80080FFFCCF8091DB018093F1008091CE
:102ED000E8008E778093E8000C945019089584B729
:102EE000877F84BF0FB6F894A895809160008861B1
:102EF00080936000109260000FBE90E080E80FB6F3
:102F0000F89480936100909361000FBE0C9450156B
:102F10000E94A2190E94FF19E2EEF0E08081846015
:102F2000808378940C94941C84E091E00C94A81411
:102F300080911B028530A9F480911B02853079F4C1
:102F40000E94A115809119028823B1F30E94621595
:102F5000882391F30E94FB170E942707EDCF0C9462
:102F6000CC15089508950C94B517292F33272330D5
:102F70003105C1F058F42130310579F022303105A6
:102F800091F582E290E02AE432E031C0213231054D
:102F9000E1F02232310501F126C082E190E02CE619
:102FA00032E025C099278130910549F028F0029739
:102FB000D1F4E8E1F2E005C0E6E4F2E002C0ECE2C0
:102FC000F2E0849190E09F0112C0672B61F489E0E8
:102FD00090E02CE532E00BC0672B29F480E490E010
:102FE0002EE732E004C080E090E020E030E0FA011B
:102FF00031832083089580E189BD82E189BD09B4D0
:1030000000FEFDCF8091D8008F7D8093D800809105
:10301000E00082608093E0008091E00081FDFCCFC1
:103020000895CF92DF92EF92FF920F931F93CF9369
:10303000DF93EC018B017A010E946F19811133C07B
:10304000E114F10439F0F70180819181081B190B1B
:10305000C80FD91FC12CD12C0115110519F1809170
:10306000E80085FD16C08091E8008E778093E80027
:10307000E114F10449F0F70180819181C80ED91E55
:10308000D182C08285E00FC00E946F19882321F38E
:103090000AC089918093F10001501109FFEFCF1A06
:1030A000DF0ADACF80E0DF91CF911F910F91FF907F
:1030B000EF90DF90CF90089520912202309123026B
:1030C0002617370748F06115710539F42091E8009B
:1030D0002E772093E80001C0B901FC0120E06115C2
:1030E000710579F180911B028823F1F18530F1F1AE
:1030F0008091E80083FD3CC08091E80082FD2EC0F5
:103100008091E80080FFEBCF2091F3008091F200E6
:1031100090E0922B6115710551F08830910538F4DB
:1031200021912093F100615071090196F3CF21E0C4
:10313000089709F020E08091E8008E778093E800FE
:10314000CECF2111CFCF0AC080911B02882361F01E
:10315000853061F08091E80083FD0AC08091E8002D
:1031600082FFF2CF80E0089582E0089583E0089521
:1031700081E008952091220230912302261737071B
:1031800048F06115710539F42091E8002E772093FD
:10319000E80001C0B901FC0120E06115710591F161
:1031A00080911B02882309F440C0853009F43FC098
:1031B0008091E80083FD3DC08091E80082FD2FC032
:1031C0008091E80080FFE9CF2091F3008091F20028
:1031D00090E0922B6115710559F08830910540F40B
:1031E00024912093F1003196615071090196F2CF3C
:1031F00021E0089709F020E08091E8008E77809325
:10320000E800CBCF2111CCCF0AC080911B028823CC
:1032100061F0853061F08091E80083FD0AC0809103
:10322000E80082FFF2CF80E0089582E0089583E015
:10323000089581E00895982F973068F59093E900FC
:10324000981739F07091EC002091ED005091F0004A
:1032500003C0242F762F50E021FD02C09F5FECCFEA
:103260003091EB003E7F3093EB003091ED003D7FDD
:103270003093ED003091EB0031603093EB007093B0
:10328000EC002093ED005093F0002091EE0027FD1C
:10329000E5CF80E008958F708093E90081E0089584
:1032A00080911C0287FF11C08091E80082FD05C05B
:1032B00080911B028111F8CF11C08091E8008B77BB
:1032C0000BC080911B02882349F08091E80080FFA9
:1032D000F8CF8091E8008E778093E80008952091E0
:1032E000E4003091E50095E64091EC00842F817078
:1032F00040FF23C08091E80080FD1DC080911B022B
:10330000882399F0853099F08091EB0085FD11C0FC
:103310004091E4005091E5002417350729F39150BE
:1033200011F09A01E1CF84E0089582E0089583E0EE
:10333000089581E0089580E008954091E80042FFFB
:10334000DDCF08950E94101A0E94181AE0EEF0E0F6
:10335000808181608083E8EDF0E080818F778083D9
:1033600019BCA7EDB0E08C918E7F8C9380818F7E0D
:10337000808310921A0208950F931F93CF93DF93C7
:103380000E94101A0E94181AC8EDD0E088818F7729
:10339000888388818068888388818F7D888319BC31
:1033A00010921B021092170210921902109218022A
:1033B00000EE10E0F80180818B7F8083888181603E
:1033C000888342E060E080E00E941B19E1EEF0E0BB
:1033D00080818E7F8083E2EEF0E080818160808357
:1033E000808188608083F80180818E7F80838881DE
:1033F00080618883DF91CF911F910F910895E8ED4F
:10340000F0E080818F7E8083E7EDF0E08081816055
:10341000808384E082BF81E080931A020C94BC19FF
:10342000E8EDF0E080818E7F80831092E2000895C5
:103430001092DA001092E10008951F920F920FB6D9
:103440000F9211242F933F934F935F936F937F932A
:103450008F939F93AF93BF93EF93FF938091E1007E
:1034600082FF0BC08091E20082FF07C08091E100E3
:103470008B7F8093E1000E94931C8091DA0080FF93
:103480001FC08091D80080FF1BC08091DA008E7F22
:103490008093DA008091D90080FF0DC080E189BD62
:1034A00082E189BD09B400FEFDCF81E080931B025B
:1034B0000E947D1605C019BC10921B020E948B163B
:1034C0008091E10080FF19C08091E20080FF15C06B
:1034D0008091E2008E7F8093E2008091E200806123
:1034E0008093E2008091D80080628093D80019BC5C
:1034F00085E080931B020E9490168091E10084FF7A
:1035000030C08091E20084FF2CC080E189BD82E15F
:1035100089BD09B400FEFDCF8091D8008F7D8093D6
:10352000D8008091E1008F7E8093E1008091E200DD
:103530008F7E8093E2008091E20081608093E200C0
:1035400080911702882311F084E007C08091E30086
:1035500087FD02C081E001C083E080931B020E94CE
:1035600098168091E10083FF29C08091E20083FFDB
:1035700025C08091E100877F8093E10082E0809305
:103580001B02109217028091E1008E7F8093E10070
:103590008091E2008E7F8093E2008091E200806162
:1035A0008093E20042E060E080E00E941B1980917D
:1035B000F00088608093F0000E948E16FF91EF91DA
:1035C000BF91AF919F918F917F916F915F914F913B
:1035D0003F912F910F900FBE0F901F9018951F9243
:1035E0000F920FB60F9211242F933F934F935F9337
:1035F0006F937F938F939F93AF93BF93CF93DF93FB
:10360000EF93FF93C091E900CF708091EC00D82F29
:10361000D17080FDD0E81092E9008091F000877FA2
:103620008093F00078940E94331B1092E9008091FF
:10363000F00088608093F000CD2BCF70C093E9003C
:10364000FF91EF91DF91CF91BF91AF919F918F91BA
:103650007F916F915F914F913F912F910F900FBE8E
:103660000F901F9018951F93CF93DF93CDB7DEB7C0
:10367000AA970FB6F894DEBF0FBECDBFECE1F2E023
:103680008091F100819322E0E432F207C9F70E94B1
:10369000B1168091E80083FF2EC180911C029091A9
:1036A0001D02492F50E04A30510508F024C1FA01AB
:1036B000EE59FF4F0C94AF1C803821F0823809F08E
:1036C0001AC108C08091180290911902992389F0BB
:1036D00082600FC0809120028F70873008F00BC18C
:1036E0008093E9008091EB0085FB882780F9109298
:1036F000E9009091E800977F9093E8008093F100B3
:103700001092F100D1C0282F2D7F09F0F4C088233A
:1037100019F0823061F0EFC080911E02813009F013
:10372000EAC0933009F080E0809319022EC08091A6
:103730001E0281112AC0809120028F702FEF280F66
:10374000263008F0D8C08093E9002091EB0020FFDC
:103750001CC0933021F48091EB00806214C09091E2
:10376000EB0090619093EB0021E030E0A90102C0F2
:10377000440F551F8A95E2F74093EA001092EA0041
:103780008091EB0088608093EB001092E9008091BB
:10379000E800877F8093E8000E945019ACC0811137
:1037A000AAC010911E021F778091E3008078812BC0
:1037B0008093E3008091E800877F8093E8000E9477
:1037C00050198091E80080FFFCCF8091E300806871
:1037D0008093E300111102C082E001C083E0809376
:1037E0001B0289C08058823008F085C080911E027B
:1037F00090911F028C3D53E0950779F583E08A8311
:103800008AE289834FB7F894DE01139620E03EE008
:1038100051E2E32FF0E050935700E49120FF03C002
:10382000E295EF703F5FEF708E2F90E0EA3010F07E
:10383000C79601C0C0968D939D932F5F243149F7A1
:103840004FBF8091E800877F8093E8006AE270E0D4
:10385000CE0101960E945C1816C060912002709102
:103860002102AE014F5F5F4F0E94B317BC01892B4D
:1038700009F441C09091E800977F9093E800898116
:103880009A810E94BA188091E8008B778093E800B3
:1038900032C0803881F58091E800877F8093E8000E
:1038A000809117028093F1008091E8008E7772CFAB
:1038B000811121C080911E0290911F0299270297C9
:1038C000D4F48091E800877F8093E80080911E0205
:1038D000809317020E94501980911702811106C02F
:1038E0008091E30087FD02C081E001C084E0809305
:1038F0001B020E94A2168091E80083FF0AC08091FB
:10390000E800877F8093E8008091EB0080628093DD
:10391000EB00AA960FB6F894DEBF0FBECDBFDF91C5
:10392000CF911F9108950895CF9380911B02882312
:10393000A1F0C091E900CF709091EC00892F8170C7
:1039400090FD80E8C82B1092E9008091E80083FD8B
:103950000E94331BCF70C093E900CF910895EE0F02
:10396000FF1F0590F491E02D0994FB01DC0104C0D8
:103970008D910190801921F441505040C8F7881B67
:10398000990B0895F999FECF92BD81BDF89A9927B8
:1039900080B50895A8E1B0E042E050E00C94F61C38
:1039A000262FF999FECF92BD81BDF89A019700B4F8
:1039B000021639F01FBA20BD0FB6F894FA9AF99A98
:1039C0000FBE08950396272F0E94D11C0E94D01C81
:1039D000252F0E94D11C242F0C94D11C0196272F37
:1039E0000E94D11C0C94D01CDC01CB01FC01F99984
:1039F000FECF06C0F2BDE1BDF89A319600B40D923B
:0C3A000041505040B8F70895F894FFCFF3
:103A0C00C800A6014A164F167B167C164D164E168C
:103A1C0001C6F437959392F6F76766363534979668
:063A2C009430333231F545
:00000001FF
